:100000008C019D018F019001910192019301940156
:1000100095019601980199019A0183161030850087
:1000200000308600640027308100831290289B01F5
:100030000C089C006D200314980203182A2803144E
:100040000130990203182A28031401309A02031878
:100050002A281B149C031C086D2003149902031802
:100060003728031401309A02031837281B149C0305
:100070001C086D2003149A02031840280314412819
:100080001B0C00349B010C089C006D20031098078A
:10009000031C5528031001309907031C5528031031
:1000A00001309A07031C55281B149C031C086D2063
:1000B00003109907031C6228031001309A07031CE0
:1000C00062281B149C031C086D2003149A07031C50
:1000D0006B2803146C281B0C003482070034003496
:1000E0000A3400340034643400340334E834003417
:1000F0002734103401348634A0340F344234403471
:1001000082073F3406345B344F3466346D347D34BB
:1001100007347F346734803482070034B134BC3410
:10012000831600308600831211308C0009308D0058
:100130008E0106309D0017200318A5288E0A8D0316
:10014000031D9B2803308C02A828422003308C0218
:1001500009308D0010301D079B009B031B08840095
:100160000E088E0180009D0301300C07031D9B28A3
:1001700018088F0097018101000000009D013C30AC
:100180008C008B0110308500831618308500831297
:100190000F301D078400000880209B0005300315E8
:1001A0001D02031DD4289B171B0886001D08000094
:1001B00085000B1DDE28970A0B11E12800000000C6
:1001C000000029309B009B0BE32800009D0A0730AC
:1001D00003111D02031DC8280000B6309B009B0BB5
:1001E000EF2800009D018C0BC82800001D309B00EB
:1001F0009B0BF828000000000B1D0129970A0B112A
:100200000429000000000000030186001030850072
:1002100083161030850083120B19970A0B11010801
:10022000990017089A009B019B0A851585110B11EF
:10023000010803111902031914299B0A9B099B0A3F
:100240001B0A980017308500831601308600831240
:10025000061C2B29852900308C20031403111A0257
:10026000031C4429031D542901308C20031103145D
:100270001902031C4429031D542902308C20031445
:100280001802031C4429542900308C208F001A08BE
:10029000930001308C2090001908940002308C20CB
:1002A000910018089500632900308C2093001A08EB
:1002B0008F0001308C2094001908900002308C20AF
:1002C000950018089100150803149102031872296B
:1002D00003140130900203187229031401308F02B5
:1002E0000318722914080314900203187C290314BC
:1002F00001308F0203187C2913088F020F089A001F
:100300001008990011089800A32902308C200310CE
:100310009807031C9529031001309907031C9529A0
:10032000031001309A07031C952901308C2003101B
:100330009907031CA029031001309A07031CA02968
:0C03400003018C209A07103085009028E3
:00000001FF
